:1070000055C000006EC000006CC000006AC00000E7
:1070100068C0000066C0000064C0000062C00000DC
:1070200060C000005EC00000F4C400005AC0000050
:1070300058C0000056C0000054C0000052C00000FC
:1070400050C0000078C000004CC000004AC00000E2
:1070500048C0000046C0000044C0000042C000001C
:1070600040C000003EC000003CC000003AC000002C
:1070700038C0000036C0000034C0000032C000003C
:1070800030C000002EC000002CC000002AC000004C
:1070900028C0000026C0000024C0000022C000005C
:1070A00020C000001EC000001CC0000011241FBE34
:1070B000CFEFDAE0DEBFCDBF11E0A0E0B1E0E6E364
:1070C000FFE702C005900D92A83AB107D9F711E089
:1070D000A8EAB1E001C01D92AE3BB107E1F792D33F
:1070E00028C78ECFF89410926F00109281001092F2
:1070F00085001092840081E085BF15BE47985D9A97
:10710000289A0C94000008952091B2013091B301A7
:107110002F5F3F4F3093B3012093B201932F37FF7E
:1071200003C08EEF831B982F990F921710F4479886
:107130000895479A08951F920F920FB60F92112447
:107140002F938F939F93EF93FF931092850010924C
:1071500084008091A8019091A901009741F00197C6
:107160009093A9018093A801892B09F45D9A8091DD
:10717000AA019091AB01009741F001979093AB0168
:107180008093AA01892B09F4289AE0E0F0E0859128
:1071900094918F5F9F4F49F08091AC019091AD0128
:1071A00001969093AD018093AC01FF91EF919F9177
:1071B0008F912F910F900FBE0F901F90189584E024
:1071C0008093E9000DC08091E8008B778093E80000
:1071D00003C08EB3882351F08091E80082FFF9CF7D
:1071E0008091E80085FFEFCF8091F1000895982FFE
:1071F00083E08093E9008091E80085FD0DC08091D7
:10720000E8008E778093E80003C08EB3882369F08E
:107210008091E80080FFF9CF9093F1005D9884E6BB
:1072200090E09093A9018093A80108954F925F92F6
:107230006F927F928F929F92AF92BF92CF92DF9286
:10724000EF92FF920F931F93CF93DF9384E080938D
:10725000E9008091E80082FF5AC2289884E690E015
:107260009093AB018093AA01AADF182F853439F4DB
:107270008CE49DE19093AD018093AC0103C0843513
:1072800019F49DDF8DE019C28C34E1F38035D1F320
:10729000843721F484E4ABDF80E00FC2813611F43F
:1072A00089E50BC28134B1F48ADF182F88DF90E0C2
:1072B000880F991FAA2797FDA095BA2F312F330F5A
:1072C00020E0442737FD4095542F822B932BA42B8D
:1072D000B52BC4C1803711F483E5EFC1833549F480
:1072E000C0E0D1E0899183DF21E0C730D207D1F738
:1072F000E5C1863521F481E37ADF80E3DEC183379F
:1073000031F487E874DF85E972DF8EE1D6C1853616
:10731000B9F4E0E0F0E093E085E090935700E89561
:1073200007B600FCFDCF80935700E89507B600FC38
:10733000FDCFE058FF4FA0E7E030FA0771F7A2CF8A
:107340008C3651F43CDF809599E0E1E0F0E0082EC6
:1073500090935700E89596CF823739F4E1E0F0E05A
:1073600089E0809357008491A8C1863439F4E0E025
:10737000F0E089E08093570084919FC18E3439F406
:10738000E3E0F0E089E080935700849196C1813575
:1073900039F4E2E0F0E089E08093570084918DC1F8
:1073A000823631F489E523DF80E021DF80E885C182
:1073B000823419F0873609F0E5C01092AD011092C1
:1073C000AC01FDDE082FFBDEF82EF9DE682E8554B9
:1073D000823008F071C1902F80E0CF2DD0E0C82B13
:1073E000D92B10926F00173609F04BC081E18093C2
:1073F0005700E895DD24CC24C3943FC0E090AE0153
:10740000F090AF010091B0011091B101B6E46B169C
:10741000D9F4ED2DF0E0EE29FF29E4918E2FE7DE7F
:10742000DD2081F082E090E0A0E0B0E0E80EF91EFF
:107430000A1F1B1FE092AE01F092AF010093B00152
:107440001093B101DC2418C0D801C701B695A795E7
:107450009795879558D5CBDE82E090E0A0E0B0E02C
:10746000E80EF91E0A1F1B1FE092AE01F092AF0159
:107470000093B0011093B1012197209709F0BECF7E
:107480007DC08090AE019090AF01A090B001B0900F
:10749000B10196E4691609F05DC083E0F4018093C0
:1074A0005700E89507B600FCFDCF54C0F6E46F1610
:1074B00061F5772031F1E090AE01F090AF010091DD
:1074C000B0011091B1017BDED82ECC24852D90E047
:1074D0008C299D29F7010C0140925700E895112451
:1074E00082E090E0A0E0B0E0E80EF91E0A1F1B1F4A
:1074F000E092AE01F092AF010093B0011093B101A0
:1075000002C05DDE582E742423C0E090AE01F090DE
:10751000AF010091B0011091B10116950795F79454
:10752000E7944DDE682FC701F6D48091AE019091AB
:10753000AF01A091B001B091B1010296A11DB11DA2
:107540008093AE019093AF01A093B001B093B101CD
:10755000219704C05524772444244394209709F0AC
:10756000A5CF96E4691641F485E0F40180935700B5
:10757000E89507B600FCFDCF8DE039DE82E0809310
:107580006F009CC0833471F40091AE011091AF0183
:1075900016DE90E021E0F8010C0120935700E895F9
:1075A000112470CE833619F5E090AE01F090AF0152
:1075B0000091B0011091B10102DEF701E16090E0AD
:1075C00021E00C0120935700E895112482E090E01F
:1075D000A0E0B0E0E80EF91E0A1F1B1FE092AE010A
:1075E000F092AF010093B0011093B1014BCE8D36F4
:1075F00061F4E091AE01F091AF0185E08093570016
:10760000E89507B600FCFDCF3DCE823551F4E09100
:10761000AE01F091AF0105911491812FE8DD802F2B
:107620004CC0843421F5E090AE01F090AF010091A0
:10763000B0011091B10116950795F794E794BFDD5D
:10764000682FC70168D48091AE019091AF01A091DD
:10765000B001B091B1010296A11DB11D8093AE01A0
:107660009093AF01A093B001B093B1010BCE8436DB
:1076700009F5E090AE01F090AF010091B0011091DA
:10768000B101D801C701B695A795979587953BD4C9
:10769000AEDD82E090E0A0E0B0E0E80EF91E0A1F47
:1076A0001B1FE092AE01F092AF010093B001109366
:1076B000B10104C08B3111F08FE399DD83E0809339
:1076C000E9009091E8008091E8008E778093E800CF
:1076D00095FF04C010C08EB38823C9F08091E800E4
:1076E00080FFF9CF8091E8008E778093E80003C097
:1076F0008EB3882361F08091E80080FFF9CF84E0A9
:107700008093E9008091E8008B778093E800DF9117
:10771000CF911F910F91FF90EF90DF90CF90BF908E
:10772000AF909F908F907F906F905F904F90089553
:107730009091B601892F8F77813249F58091B701F9
:107740008032A1F0813219F5913A09F58091E80073
:10775000877F8093E8008DE091E067E070E00AD2D7
:107760008091E8008B778093E8000895913279F456
:107770008091E800877F8093E8008DE091E067E0EA
:1077800070E05CD28091E8008E778093E8000895E5
:1077900082E061EC42E0B4D083E061E842E1B0D045
:1077A00084E060E842E1ACC084B7877F84BF88E1B1
:1077B0000FB6F89480936000109260000FBE20E82E
:1077C00080E090E00FB6F894209361008093610010
:1077D0000FBE81E085BF92E095BF3F9A209A559AEF
:1077E000E1E6F0E02083108247985D9A289A109293
:1077F00089008AEF8093880090936F0083E08093E4
:107800008100EFC01F9388E10FB6F8948093600069
:10781000109260000FBE84B714BE182F10FF08C06E
:10782000E0E0F0E0859194918F5F9F4F09F05ADC82
:107830002091000A3091010A1092010A1092000A68
:1078400013FF0FC08091090190910A012817390791
:1078500041F0E0E0F0E0859194918F5F9F4F09F057
:1078600041DCA2DF78941092AD011092AC010CC003
:10787000DDDC37D38091AC019091AD0181549F4103
:1078800010F01092140140DC80911401882381F7DC
:107890008091E00081608093E00024DC80E090E053
:1078A0001F910895FA01923049F0933061F09130C0
:1078B000F9F485E191E022E130E01EC087E291E039
:1078C0002EE330E019C0882329F485E691E024E016
:1078D00030E012C0813029F489E691E022E230E004
:1078E0000BC0823029F48DE891E028E130E004C03B
:1078F00080E090E020E030E091838083C90108952A
:107900008093E9008091EB0081608093EB001092FE
:10791000ED006093EC004093ED008091EE00881F35
:107920008827881F08958091B60188238CF403C0AE
:107930008EB38823B1F08091E80082FFF9CF809167
:10794000E8008B778093E80008958EB3882349F090
:107950008091E80080FFF9CF8091E8008E778093D6
:10796000E8000895EF92FF920F931F9345D04CD0FB
:1079700008ED10E0F80180818F7780838081806836
:10798000808380818F7D808319BC1EBA1092B401E0
:1079900080EEE82EF12CF70180818B7F8083F80147
:1079A00080818160808380E060E042E0A9DFE1EED9
:1079B000F0E080818E7F8083E2EEF0E08081816064
:1079C0008083808188608083F70180818E7F8083BF
:1079D000F8018081806180831F910F91FF90EF906B
:1079E0000895E7EDF0E08081816080838AE482BFC2
:1079F00081E08093B501B6CFE8EDF0E080818E7F25
:107A000080831092E20008951092DA001092E10053
:107A100008951F920F920FB60F9211242F933F9348
:107A20004F935F936F937F938F939F93AF93BF9386
:107A3000EF93FF938091DA0080FF1BC08091D80004
:107A400080FF17C08091DA008E7F8093DA008091EA
:107A5000D90080FF0BC080E189BD82E189BD09B4F6
:107A600000FEFDCF81E08EBB3BD203C019BC1EBA25
:107A700037D28091E10080FF17C08091E20080FF43
:107A800013C08091E2008E7F8093E2008091E2003B
:107A900080618093E2008091D80080628093D8005A
:107AA00019BC85E08EBB1CD28091E10084FF2CC004
:107AB0008091E20084FF28C080E189BD82E189BD18
:107AC00009B400FEFDCF8091D8008F7D8093D8004F
:107AD0008091E1008F7E8093E1008091E2008F7EB3
:107AE0008093E2008091E20081608093E2008091C7
:107AF000B401882331F48091E30087FD02C081E066
:107B000001C084E08EBBECD18091E10083FF21C0F5
:107B10008091E20083FF1DC08091E100877F809308
:107B2000E10082E08EBB1092B4018091E1008E7F73
:107B30008093E1008091E2008E7F8093E20080914B
:107B4000E20080618093E20080E060E042E0D8DE05
:107B5000C7D1FF91EF91BF91AF919F918F917F918D
:107B60006F915F914F913F912F910F900FBE0F90AA
:107B70001F9018959C014091BC015091BD01461782
:107B8000570718F4F90190E044C06115710511F030
:107B9000AB01F8CF8091E8008E778093E80040E059
:107BA00050E0F0CF8EB3882309F444C0853009F447
:107BB00043C08091E80083FF02C081E00895809176
:107BC000E80082FD31C08091E80080FF22C08091F2
:107BD000F3009091F200782F60E0292F30E0262BFF
:107BE000372B07C081918093F100415050402F5FA7
:107BF0003F4F4115510519F02830310598F390E0B9
:107C00002830310509F491E08091E8008E77809367
:107C1000E8004115510531F6992321F605C08EB3D0
:107C2000882341F0853041F08091E80082FFF7CF52
:107C300080E0089582E0089583E008959C01611535
:107C4000710529F48091E8008B778093E800F901B1
:107C500026C08EB3882391F1853091F18091E800A0
:107C600083FF02C081E008958091E80082FFF1CF98
:107C700006C08091F10081936150704059F02091CD
:107C8000F3008091F200322F20E090E0822B932BC2
:107C9000892B79F78091E8008B778093E800611554
:107CA0007105B9F605C08EB3882341F0853041F0E7
:107CB0008091E80080FFF7CF80E0089582E008958A
:107CC00083E008950F931F93DF93CF9300D0CDB738
:107CD000DEB7E6EBF1E08091F100819381E0EE3BCD
:107CE000F807C9F725DD8091E80083FFE4C08091A3
:107CF000B6019091B701953009F46DC0963040F40B
:107D0000913081F1913070F0933009F0D4C02AC0E5
:107D1000983009F4A3C0993009F4B2C0963009F044
:107D2000CAC07CC0803809F4C6C0823809F0C3C01C
:107D30008091BA0187708093E9008091EB001092E6
:107D4000E9002091E800277F2093E80090E025E0FB
:107D5000969587952A95E1F781708093F1001092AE
:107D6000F10087C0882319F0823009F0A4C08F7118
:107D7000823009F0A0C08091B801882331F52091AC
:107D8000BA01277009F497C02093E9008091EB00B5
:107D900080FF1BC0933021F48091EB00806213C000
:107DA0008091EB0080618093EB0081E090E002C065
:107DB000880F991F2A95E2F78093EA001092EA0053
:107DC0008091EB0088608093EB001092E900809135
:107DD000E800877F51C0882309F06DC01091B80179
:107DE0001F770FB7F8948091E800877F8093E800B1
:107DF0009ADD8091E80080FFFCCF8091E3008078DD
:107E0000812B8093E30080688093E300112311F4B9
:107E100082E001C083E08EBB0FBF4DC0805882302E
:107E200008F049C08091B8019091B9016091BA0100
:107E3000AE014F5F5F4F36DDBC01009709F43BC0D8
:107E40008091E800877F8093E80089819A8192DEA3
:107E50008091E8008B778093E8002DC0803859F539
:107E60008091E800877F8093E8008091B40180933F
:107E7000F1008091E8008E778093E80054DD1BC00C
:107E80008823C9F49091B8019230A8F48091E80059
:107E9000877F8093E8009093B40145DD8091B40121
:107EA000882331F48091E30087FD02C081E001C0A6
:107EB00084E08EBB6DDC8091E80083FF0AC0809176
:107EC000EB0080628093EB008091E800877F8093D5
:107ED000E8000F900F90CF91DF911F910F910895BF
:107EE00008951F938EB3882361F01091E9001092DA
:107EF000E9008091E80083FF01C0E4DE1770109371
:107F0000E9001F910895F999FECF92BD81BDF89ABD
:107F1000992780B50895262FF999FECF1FBA92BDF3
:107F200081BD20BD0FB6F894FA9AF99A0FBE01965A
:067F30000895F894FFCF54
:107F36004341544552494E41007777000A000000FC
:107F4600000000080112011001020000084123018F
:107F56000701000201000109023E00020100803211
:107F66000904000001020201000524001001042496
:107F760002040524060001070582030800FF090420
:107F86000100020A000000070504021000010705AF
:107F960083021000010403090422034100720064F5
:107FA60000750069006E006F0020004C0065006FD0
:107FB600006E006100720064006F0000001803414B
:107FC6000072006400750069006E006F0020004CAE
:087FD600004C00430000000014
:040000030000700089
:00000001FF
